:100000004FC0FECFFDCFFCCFFBCFFACFF9CFF8CF5B
:10001000F7CFF6CFF5CFF4CFF3CFF2CFF1CFF0CFCC
:10002000EFCFEECFEDCF1027E80364000A00010008
:100030000010000110000100253032642E253031FF
:100040006456202843432920253031642E25303240
:10005000644100253032642E253031645620284317
:10006000562920253031642E253032644100253058
:1000700032642E253031645720426F61726420460D
:10008000726565007777772E426F6172644672659C
:10009000652E6B72000080C002008B01960000008C
:1000A000F894EE27ECBBF1E0FBBFEBBFE5BFF8E156
:1000B000F1BDE1BD8DE0A2E0BB27ED938A95E9F7A4
:1000C00080E094E0A0E6ED930197E9F7E8E9F0E03D
:1000D00085919591009761F0A591B5910590159046
:1000E000BF01F00105900D920197E1F7FB01F0CF00
:1000F000EFE5EDBFE4E0EEBFC0E6D1E00DC0E88182
:10010000E06CE7B98DE08A95F1F7369A349BFECF23
:10011000349AE4B1F5B1F4C1E0E0E8BBE7BBE5BB7C
:10012000E4BBE2BBE1BBE3BFE2BFEFBDEEBDEDBDB3
:10013000ECBDE7BDE6BDEBBDEABDE9BDE8BDE2BD96
:10014000E5BDE4BDE3BDE5BFE9BFEAB9E0E8E8B974
:10015000E0E0E0BFE0ECE7B9E2E8E6B9E0E0EDB905
:10016000E6BFE0E1EA93A0D151D3C9DF3F01D3015B
:1001700050D3ADD43F018614970490F4F301E819ED
:10018000F9094AD310F443010AC04BD340F0E0917F
:100190006201EF5FE0936201E0E0E093630114C06D
:1001A0006814790488F4F401E619F70935D310F4DA
:1001B00043010AC036D340F0E0916301EF5FE09362
:1001C0006301E0E0E0936201A0916201A43130F0AC
:1001D000F40131964F01E0E0E0936201A0916301E8
:1001E000A43148F0082C092819F0F40131974F0187
:1001F000E0E0E0936301E1E0EA9381DF3F01F30196
:1002000066277727D4D3DF01CB01E0E0F0E060E29E
:1002100070E4FBD393D33F01FCD26E167F0620F02F
:10022000F30133973F0106C0F4D26E167F0610F437
:1002300066247724A614B70490F4F301EA19FB09A5
:10024000EBD210F453010AC0ECD240F0E091660109
:10025000EF5FE0936601E0E0E093670114C06A1489
:100260007B0488F4F501E619F709D6D210F453019E
:100270000AC0D7D240F0E0916701EF5FE0936701D9
:10028000E0E0E0936601A0916601A43130F0F50151
:1002900031965F01E0E0E0936601A0916701A4312F
:1002A00048F00A2C0B2819F0F50131975F01E0E0C6
:1002B000E0936701D401B9D20AD4E0936001D4017C
:1002C000B4D218D4E0936101D501E4E6F0E0FFD3A5
:1002D000E0936401D501E4E6F0E00CD4E09365011D
:1002E000082C092819F00A2C0B2809F413C0F50171
:1002F000D401E5D3DF01E4E6F0E0E9D36F01D601F4
:1003000094D2E5D3E0936801D6018FD2F3D3E09382
:10031000690105C0E0E0E0936901E0936801B099EC
:1003200004C086D2E8E3F0E005C0B09B14C080D2E0
:10033000E3E5F0E0FA93EA93E09160017ED2E09188
:1003400061017BD2E091640178D2E091650175D2C0
:1003500080E11CD264965AD259D258D069D295D035
:10036000E0916801E03021F4E0916901E03071F042
:100370005FD2EEE6F0E066D2E09168015ED2E091F5
:1003800069015BD288E002D22C9607C051D2E4E822
:10039000F0E058D280E0FAD1249638D2E1E0EA9336
:1003A00035D046D272D041D250D2DECEFFCFE881D6
:1003B000E07111F0949A01C09498E881E07211F014
:1003C000959A01C09598E881E07411F0969A01C061
:1003D0009698E881E07811F0979A01C0979883E0A9
:1003E0008A95F1F7929A87E08A95F1F7929887E0DB
:1003F0008A95F1F785C0E8812AD2E881E295E88301
:10040000E88125D283E48A95F1F77AC0E881F0E0AB
:10041000E557FE4FE081A981EA0F1BD2E981E09305
:100420008F01E881E093900122960895E2E011D2D5
:10043000F0D10BD2ECE00DD2E1E00BD2EAD105D243
:10044000E0E0E0939001E0938F010895A881AA3045
:1004500031F0E0919101A0918F01AE1760F0D6D1FB
:10046000E0919001EF5FE0939001EA93CFDFA881E4
:10047000AA3009F445C0E0918F01EF5FE0938F014E
:10048000909AE881E6D190983BC01A93A981BA81ED
:10049000ED91A983BA831E2FE03019F01A93D6DFAD
:1004A000F5CF1881239608958C9A8D9A8E9A8F9AFB
:1004B0008A9A889A899A929890989198E881E0937C
:1004C0009101E058E0938D01E881E054E0938E01C2
:1004D000E4E1F0E0BAD1E0E3BAD1BDD1BCD185E826
:1004E0008A95F1F7E0E2B3D185E88A95F1F7E8E281
:1004F000B0D1E4E0AED1E5E8ACD1E6E0AAD196DF38
:10050000219608950BD3ACD11296F7D23097F1F023
:10051000A7D1A9D18F01309761F00230E0E01E072A
:10052000A0F0F80131978F01AA81BB811496ED9359
:10053000FC9396D112969AD13197AC81A08390D139
:10054000DCD2FF2312F08CD191D105C089D1EFEF1D
:10055000FFEFED93FC93E9D2259608952697DAD222
:1005600010E0AC85BD85E0E0F0E0ED93FC93EA8916
:10057000FB893196EA8BFB8B3197E4912E2FE0308B
:1005800009F4FEC0E12FE03031F4253211F411E01E
:1005900001C072D1F4C0E130A1F4253211F46CD164
:1005A000EDC012E040E000E02D3211F401E0E7C0C0
:1005B0002B3211F44BE2E3C0203211F440E2DFC0F1
:1005C00002C0E23039F450E013E0203311F4006847
:1005D000D6C003C0E33009F0D2C0203310F02A3374
:1005E00008F007C0AAE05A9F502DE22FE0535E0F9B
:1005F000C6C0E22FE33639F447D149D145D1A481B1
:10060000AA9349D1BBC0E33731F44CD14DD14FD17E
:10061000E8D01E2F08C0E03751F444D145D147D16E
:10062000EAD01E2F086002600F7730E02EC0E4365B
:1006300011F0E93611F4046002C0E53729F4E6E26E
:10064000F0E038D115E00BC0E83511F4086003C0C4
:10065000E83709F093C0E0E3F0E02CD114E002FFAA
:1006600011C020D121D129D1AB85AA232AF4EA8552
:10067000FB8514D222D14DE2403011F01F5F01C042
:100680000B7F03C00FD110D118D100FD10C015177A
:1006900070F407FF08C002FF04C00B7F242F115025
:1006A00001C020E301C020E2E7D05150F0CF312F4C
:1006B00001FF15C0303091F003FF05C0EE81FF81CE
:1006C0002591F8D005C0AE81BF812D91AE83BF8347
:1006D000D3D0503009F051503150ECCF46C020E318
:1006E000EE81FF810ED2E887F987EE81FF81329695
:1006F000E1D0E885F985AA85BB85AE17BF0748F02C
:100700002F5FA885B985EA85FB85EA1BFB0BD5D051
:10071000F0CF2A3328F003FF02C0295F01C0295D12
:1007200004FD19C0213320F4A885B985119709F477
:1007300009C0531710F000FF01C011C020E207FFED
:100740000AC020E3006102FF06C00B7F4A93A3D0DA
:10075000503009F0515090D0503009F05150315084
:10076000A885B985129708F0BACF00FF07C05030AE
:1007700029F05150E0E2EA938ED0F9CF10E0F7CEA5
:10078000AC85BD85BAD1CDD164960895FF92F82E7F
:100790002697C2D195D0309719F4EFEFFFEF1DC027
:1007A000DE01169677D18D018BD084D0E0E0E8870A
:1007B000E987DE011A966ED1A0D144D01A930A932C
:1007C000E2E8F2E03FD0FE013A963CD0C7DE9F015E
:1007D000AE81BF81E0E0EC93F901A5D12A96FF90AC
:1007E0000895A991B991EE27FF276D91662311F025
:1007F0003196FBCF0895AA27BB27E991F99105907F
:10080000002011F01196FBCFFD010895E0E0EA937E
:100810000895E3E0F0E008952F01FBDFE415F5050E
:100820000895F7DFE415F5050895EAE0F0E008958E
:10083000EAE6F1E0FA93EA930895FF27662777271F
:1008400064D10895FA93EA930895FCDF3EC0EA93D9
:10085000AECDEA93D0CD85E88A95F1F7E0E3F7CF06
:10086000AA81BB810895149648D10895ED91FD9118
:100870003196FE93EE9308952A93ED85FE85E2DF8F
:10088000E989FA8909950895E889F98908953497DD
:10089000E88BF98B0895ED85FE85D4DFE989FA8927
:1008A00009950895F1DFF3CFA889B989DCCFEE83EC
:1008B000FF83C8CFEE83FF830895EA87FB870895FF
:1008C000DE011C96E7D019D10895E991F99130968F
:1008D00039F088EE93E00197F1F7A8953197C9F7C1
:1008E0000895552342F4503811F4E0FF04C03196C6
:1008F000691F791F6BF050E8572711F45F9373C09D
:100900005F3F31F0660F000C57956795752F08957E
:100910005F9300200AF073C06CC050E8192E1522B6
:10092000880F991F9527550F879550E8072E0522A8
:10093000660F771F7527550F67950895689401C056
:10094000E8945F93F2DF703818F07F3F08F44BC0F3
:1009500056E1571BAAF4519558300EF4593030F037
:10096000EFEFFFEF6FEF7FE777F91AC07727552397
:10097000B9F0EE0FFF1F661F771F5A95D1F710C011
:100980007727583028F0EF2FF62F672F5850F9CFE0
:10099000552331F076956795F795E7955A95D1F7F8
:1009A00000200AF47FD05F910895689401C0E89414
:1009B000309760407040B1F0002426F0772312F4A5
:1009C000009470D0172E7EE1112032F07A95EE0F50
:1009D000FF1F661F111CF9CFEF2FF62F612D5F93BC
:1009E0008ADF5F910895EE27FF27662777275F91BB
:1009F0000895EFEFFFEF6FE77FEF5F910895EFEF5F
:100A0000FFEF6FE77FE75F9108955F9386DF7038B0
:100A100021F411200AF4EDCFF2CF903809F4E3CF9E
:100A200001240894970B1BF4D4F30020F3CF792F03
:100A30001F932F933F934F9311241127222733277E
:100A40004427552790E2AE17BF078607410730F0CD
:100A5000AE1BBF0B860B410B089401C08894551F39
:100A6000221F331F111CAA1FBB1F881F441F9A95EA
:100A700051F7F901612D4F913F912F911F916623FD
:100A800032F0550FEE1FFF1F661F7A9543F229DFE4
:100A90005F9108950024AF0DB01D0895F195E19583
:100AA000F0400895F09560957095E195FF4F6F4F78
:100AB0007F4F08956F2F660F660B762F0895FA9F6C
:100AC000F02DEB9FF00DEA9FE02DF10D089500242D
:100AD000112490E1AA0FBB1F001C111C0E1A1F0A43
:100AE00018F40E0E1F1E01C0A1609A9599F7FD0122
:100AF000D0010895ECDFFD010895ED91FC9111976F
:100B000008950590F491E02D08957A936A93FA93ED
:100B1000EA9308955A934A933A932A931A930A931D
:100B200008955D814C813B812A8119810881089556
:00000001FF
